:100000000C9473060C9490060C9490060C94900635
:100010000C9490060C9490060C9490060C94900608
:100020000C9490060C9490060C947E2A0C94502B01
:100030000C94B2240C9490060C9490060C949006A8
:100040000C9490060C9490060C9490060C949006D8
:100050000C9490060C943A250C9490060C949006FF
:100060000C9490060C9490060C9490060C949006B8
:100070000C9490060C9490060C9490060C949006A8
:100080000C9490060C9490060C9490060C94900698
:100090000C9490060C9490060C9490060C94900688
:1000A0000C9490060C9490060C9490064D0B4D0BFE
:1000B000790B790BE10BFF0B170D170D0A0CA30C35
:1000C000B40CB40CDC20CA20E320552090219021F0
:1000D000C72090219021102190212421702190216E
:1000E0009021902190214421902190214121902123
:1000F000FC20902190218A218A218A218A218A212B
:100100008A218A218A218A218C219021DC20BF200A
:100110009021902190219021902190219021902157
:10012000902190218C2190219021C720902188211D
:100130008821882188218821882188218821882177
:100140008C21BD2BE42BDC2CE42BDC2C302C532C11
:10015000DC2CAA2CB92C14001A000800150017007A
:1001600000001C0018000C00120013000400160010
:10017000070009000A0000000B000D000E000F0030
:1001800033001D001B00060019000500E0001100EF
:10019000100036003700380029002B00E300E10092
:1001A0002A00E2002C0001512D00340028001E021C
:1001B0001F0252002F02300200004B0024002500D5
:1001C000260025022002500051004F0021020000AD
:1001D0004E002100220023002E022F0030002602B4
:1001E00027022402E00035001E001F00200031001D
:1001F00002534900E300E1002A00E2002C00010064
:10020000370027002E0049004A0052004D004B00E5
:100210000000520040004100420043004C005000EA
:1002200051004F004E00000051003D003E003F00D5
:1002300044000000A90000000000005CE000000095
:100240003A003B003C0045000000AA00E300E1004A
:100250002A00E2002C0010504600470048004445A8
:100260004255473A2064697361626C65642E0A00E6
:1002700044454255473A20656E61626C65642E0ABA
:100280000000000000000000002A2B2800000000F1
:100290000000000000000000000000002900000035
:1002A000002C1E3420212224342627252E362D37DB
:1002B00038271E1F202122232425263333362E37AC
:1002C000381F0405060708090A0B0C0D0E0F101144
:1002D00012131415161718191A1B1C1D2F31302351
:1002E0002D350405060708090A0B0C0D0E0F101119
:1002F00012131415161718191A1B1C1D2F3130351F
:100300004C000000000000000000000000000000A1
:1003100000000000000000000000000000000000DD
:1003200000000000007E0F00D4FFFFFFC7000000A8
:10033000780A0025303258006C65645F7461736B15
:100340003A20004F6E6573686F743A206163746978
:1003500076653A2025640A000A00253031366200AD
:100360003A200025303258000A722F632030313293
:10037000333435363738394142434445460A00293B
:100380000A002575002F002575005D2800256400F2
:100390002000256400200025640020002564007CE6
:1003A0000025303258006D6F7573656B6579205B81
:1003B00062746E7C782079207620685D2872657082
:1003C0002F61636C293A205B00556E69636F646529
:1003D00020696E707574206D6F646520736574207C
:1003E000746F3A2025750A00556E69636F64652045
:1003F000696E707574206D6F646520696E69742014
:10040000746F3A2025750A00313A0964656C617988
:10041000282A31306D73293A2025750A323A096944
:100420006E74657276616C286D73293A2025750AA1
:10043000333A096D61785F73706565643A2025759C
:100440000A343A0974696D655F746F5F6D61783A5B
:100450002025750A353A09776865656C5F6D6178A6
:100460005F73706565643A2025750A363A097768C6
:1004700065656C5F74696D655F746F5F6D61783A17
:100480002025750A00703A097072696E74207661D1
:100490006C7565730A643A097365742064656661F6
:1004A000756C74730A75703A092B310A646E3A09D7
:1004B0002D310A6C743A092B31300A72743A092DC5
:1004C00031300A4553432F713A09717569740A0A2C
:1004D0007370656564203D2064656C7461202A201A
:1004E0006D61785F7370656564202A20287265707D
:1004F000656174202F2074696D655F746F5F6D6135
:1005000078290A77686572652064656C74613A20A1
:10051000637572736F723D25642C20776865656C16
:100520003D25640A53656520687474703A2F2F6501
:100530006E2E77696B6970656469612E6F72672FC3
:1005400077696B692F4D6F7573655F6B6579730A9A
:10055000004D3E20004D25753A25733E20003F0A90
:10056000003D2025750A003F0A0064656661756CD0
:1005700074730A0025750A003F0A000A092D2056E7
:10058000616C756573202D0A00710A000A092D201F
:100590004D6F7573656B6579202D0A003F00433EF2
:1005A00020004C25640A000A092D205374617475DB
:1005B00073202D0A686F73745F6B6579626F617267
:1005C000645F6C65647328293A20253032580A6BC1
:1005D0006579626F6172645F70726F746F636F6C64
:1005E0003A20253032580A6B6579626F6172645F18
:1005F00069646C653A20253032580A6B65796D6103
:10060000705F636F6E6669672E6E6B726F3A20253E
:100610003032580A74696D65725F72656164333295
:1006200028293A202530386C580A000A092D20560E
:10063000657273696F6E202D0A5649443A203078EE
:100640003132303928546563686E6F6D616E63793D
:1006500029205049443A20307841314535284174A9
:100660007265757329205645523A20307830303003
:10067000380A4255494C443A2020284665622032C7
:10068000372032303232290A4F5054494F4E533AB4
:10069000204C554641204D4F5553454B455920451B
:1006A000585452414B455920434F4E534F4C4520CF
:1006B000434F4D4D414E44204E4B524F2034303924
:1006C000360A4743433A20352E342E3020415652C5
:1006D0002D4C4942433A20322E302E302041565282
:1006E0005F415243483A20617672350A000A092D6B
:1006F00020436F6E736F6C65202D0A4553432F7135
:100700003A09717569740A6D3A096D6F7573656B95
:1007100065790A000A092D204D61676963202D0A59
:10072000443A094465627567204D65737361676576
:1007300020546F67676C650A583A094D6174726995
:1007400078204465627567204D6F646520546F673B
:10075000676C65202D2053686F77206B6579707208
:10076000657373657320696E206D6174726978209A
:10077000677269640A4B3A094B6579626F6172640A
:1007800020446562756720546F67676C65202D2073
:1007900053686F77206B657970726573732072652B
:1007A000706F72740A4D3A094465627567204D6F27
:1007B00075736520546F67676C650A563A0956650C
:1007C0007273696F6E0A533A095374617475730AD0
:1007D000433A09416374697661746520436F6E73AF
:1007E0006F6C65204D6F64650A46312D4631303A95
:1007F0000953776974636820746F204C617965725E
:1008000020302D392028463130203D204C30290A17
:10081000302D393A0953776974636820746F204C1E
:100820006179657220302D390A47524156453A099F
:1008300053776974636820746F204C617965722006
:10084000302028616C7465726E617465290A423AC1
:10085000094A756D7020746F20426F6F746C6F6100
:100860006465720A4553433A094A756D7020746F86
:1008700020426F6F746C6F616465722028616C74C4
:1008800065726E617465290A453A095072696E7421
:1008900020454550524F4D2053657474696E6773FF
:1008A0000A4253504143453A09436C656172204501
:1008B0004550524F4D0A4E3A094E4B524F20546FFD
:1008C00067676C650A006B65796D61705F636F6E59
:1008D0006669672E7261773A20253032580A2E7386
:1008E0007761705F636F6E74726F6C5F636170735A
:1008F0006C6F636B3A2025750A2E636170736C6FA1
:10090000636B5F746F5F636F6E74726F6C3A2025F8
:10091000750A2E737761705F6C63746C5F6C6775BA
:10092000693A2025750A2E737761705F7263746C63
:100930005F726775693A2025750A2E737761705F5B
:100940006C616C745F6C6775693A2025750A2E734B
:100950007761705F72616C745F726775693A2025A8
:10096000750A2E6E6F5F6775693A2025750A2E73BA
:100970007761705F67726176655F6573633A2025A2
:10098000750A2E737761705F6261636B736C61735C
:10099000685F6261636B73706163653A2025750AF5
:1009A0002E6E6B726F3A2025750A0064656275675A
:1009B0005F636F6E6669672E7261773A2025303209
:1009C000580A2E656E61626C653A2025750A2E6D97
:1009D00061747269783A2025750A2E6B6579626FA9
:1009E0006172643A2025750A2E6D6F7573653A2021
:1009F00025750A006565636F6E6669673A0A646506
:100A00006661756C745F6C617965723A2025750A50
:100A1000003F004E4B524F3A206F66660A004E4B25
:100A2000524F3A206F6E0A000A6D6F7573653A2057
:100A30006F66660A000A6D6F7573653A206F6E0AFD
:100A4000000A6B6579626F6172643A206F66660AAC
:100A5000000A6B6579626F6172643A206F6E0A00FA
:100A60000A6D61747269783A206F66660A000A6DD1
:100A700061747269783A206F6E0A000A6465627563
:100A8000673A206F66660A000A64656275673A20F5
:100A90006F6E0A000A0A4A756D70696E6720746F7E
:100AA00020626F6F746C6F616465722E2E2E200051
:100AB000433E2000436C656172696E672045455076
:100AC000524F4D0A000A002530325820006B6579DC
:100AD000626F6172645F7265706F72743A20006455
:100AE000656C5F6B65795F6269743A2063616E273C
:100AF000742064656C3A20253032580A00616464C1
:100B00005F6B65795F6269743A2063616E27742058
:100B10006164643A20253032580A005B735D005BE3
:100B2000575D005B535D005B525D005B445D005BA5
:100B3000435D000E03410074007200650075007390
:100B4000000000180354006500630068006E006F29
:100B5000006D0061006E006300790000000403096D
:100B60000409025B00030100A0FA0904000001036C
:100B70000101000921110100012240000705810344
:100B8000080001090401000103000000092111010E
:100B9000000122B6000705820320000109040200BB
:100BA00002030000000921110100012222000705B3
:100BB0008303200001070503032000011201000246
:100BC000000000080912E5A1080001020001063139
:100BD000FF0974A1010975150026FF00952075080D
:100BE00081020976150026FF00952075089102C044
:100BF00005010902A10185020901A10005091901E8
:100C000029081500250195087501810205010930A3
:100C100009311581257F95027508810609381581EE
:100C2000257F950175088106050C0A380215812576
:100C30007F950175088106C0C005010980A1018565
:100C40000319012AB700150126B700950175108117
:100C500000C0050C0901A101850419012AA0021593
:100C60000126A002950175108100C005010906A1A9
:100C7000018506050719E029E71500250195087586
:100C80000181020507190029EF1500250195F0756E
:100C90000181020508190129059505750191029543
:100CA0000175039101C005010906A101050719E0BD
:100CB00029E7150025019508750181029501750840
:100CC00081010507190029FF150026FF009506750B
:100CD00008810005081901290595057501910295FE
:100CE0000175039101C011241FBECFEFDAE0DEBF12
:100CF000CDBF11E0A0E0B1E0E4E3FBE502C0059068
:100D00000D92A63FB107D9F723E0A6EFB1E001C0ED
:100D10001D92A132B207E1F70E946D190C94982D33
:100D20000C940000FF93EF93E091F601F091F7012E
:100D3000309709F00995EF91FF910895FC01859195
:100D4000803011F0EFDFFBCF0895FF27E0E230E2C3
:100D500047FF0CC0419597FF09C0EDE26095709583
:100D600080959095611D711D811D911D27FF02C009
:100D7000219530E350E2AA27660F771F881F991F3D
:100D8000AA1FA41710F0A41B63955A95A9F7AA30BF
:100D900008F0A95FA05DAF93F3956115710581051A
:100DA000910541F7ED3211F4EF93F395F21718F432
:100DB0003F93F395FBCF8F91B5DFFA95E1F7089557
:100DC000E991F9918591803021F0853219F0AADFFF
:100DD000F9CF089520E0E89455915532C1F350338E
:100DE00011F4689455915A3348F4505390F3220FFC
:100DF000022E220F220F200D250FF4CF0EF4219585
:100E000089919991533619F3533729F1533559F193
:100E1000BC0188279927E8945C3621F4899199913F
:100E200068945591543639F446EF7EF077FF0DC043
:100E30008FEF9FEF0AC055374AE039F0583540E14F
:100E400021F0523642E009F00895FF93EF937DDFE1
:100E5000EF91FF91B7CFFF93EF93FC018191803029
:100E6000B9F360DFFBCFFF93EF9368DFF1CFDF9340
:100E7000CF93CDB7DEB72596A3DFCF91DF9108954D
:100E80009C013A9521153F4130F5BC0166277270EF
:100E9000AC01442754709C012227387094FF0FC086
:100EA00090FF02C080E101C080E0672B09F0806202
:100EB000452B09F08064232B79F080680895892FF1
:100EC0008170672B09F08260452B09F08460232B29
:100ED00019F08860089580E00895CF93DF93EB01C7
:100EE0000E944007FE01DF91CF910994CF93DF93D9
:100EF000EC01805E9109089710F0209719F464E0E6
:100F00007BE002C06FE87DE0CE010E946D078C2F70
:100F1000DF91CF910C94CD09CF93DF93EC010E9428
:100F20007C0ACE01805E9109089710F0209719F491
:100F30006BE07BE002C066E97DE0CE01DF91CF91FE
:100F40000C946D07CF93DF93EC010E947607C933B1
:100F5000D10549F42FEF87EE93E021508040904077
:100F6000E1F700C00000CE01DF91CF910C948C0717
:100F700081E0089581E008950C94BA0708950C94D7
:100F8000BE071F93CF93DF9300D000D01F92CDB741
:100F9000DEB749835A836B833091F90189819A8145
:100FA000311114C0662359F0222349F00E94620FC8
:100FB000182F682F89819A810E940B0F03C00E940D
:100FC000360F182F69817A81812F04C00E94620F29
:100FD00069817A810F900F900F900F900F90DF91A1
:100FE000CF911F910C94AB16FC01262F40815181AB
:100FF0006281738184810C94C10781E00895CF934D
:10100000DF93EC0160E00E94F407BE01DF91CF9115
:101010000C94BF070C941E180C941A1808950E9483
:10102000B50D0E940E082FEF84E39CE02150804014
:101030009040E1F700C000000C9460250F931F93CF
:10104000CF93DF938C0161E00E94F407EC01B801BB
:101050000E94BC07882309F462C0B801CE010E9437
:101060007A1D882309F45BC0B801CE010E949D223D
:10107000882309F454C0B801CE010E94961D88232C
:1010800009F44DC0B801CE010E94F921882309F46A
:1010900046C0F80182818823D9F1CF3D8CE5D8077D
:1010A00079F140F4C115FCE5DF0791F0C130DC4572
:1010B00091F02EC0CC35EDE5DE0741F1CD35FDE5F3
:1010C000DF0709F1CB35DD4519F50E94FC1320C07F
:1010D0000E940F0824C08091AC02C82FC095C17037
:1010E000C0FB80F98093AC02CC2329F080E792E02A
:1010F0000E949E0614C08EE592E00E949E0610C0DB
:101100000E94AA140CC00E94F31302C00E94FF1395
:10111000C801DF91CF911F910F910C94B807C0E0E7
:101120008C2FDF91CF911F910F9108950E949424ED
:101130000C9444090E9447090C949A24DF92EF9280
:10114000FF920F931F93CF93DF93E82FF0E0EF57B9
:10115000FD4FD490282F26952695269530E0F9014D
:10116000EF5DFC4F0491877010E0082E02C01595CA
:1011700007950A94E2F701701127F901EF5EFC4F21
:10118000E490F12C082E02C0F594E7940A94E2F75B
:1011900091E0E922FF24F901EF5FFC4FC491D0E018
:1011A00002C0D595C7958A95E2F7C170DD27011574
:1011B000110519F081EE0E94CD09E114F10419F036
:1011C00086EE0E94CD098D2D0E94FB0AEF2819F0B2
:1011D00086EE0E947C0A012B19F081EE0E947C0AA7
:1011E000CD2B51F08CE2DF91CF911F910F91FF90A9
:1011F000EF90DF900C94FB0ADF91CF911F910F913C
:10120000FF90EF90DF900895982F9F709A5096303E
:1012100010F0805D01C0895A0C949E088295982F29
:10122000937344E0949F900111248C7C869586955D
:10123000282B822F8575880F2A7A2695822B089570
:10124000CF93DF93D92F0E940E09C82F8D2F0E94B4
:101250000E092C2F30E0322F2227A901482BCA017A
:10126000DF91CF91089508950C94330981E008959A
:101270000C9436090895CF93C82F0E9434098C2FFF
:101280000E943809CF91089580E00C943B090E9498
:10129000F9220C943B09CF930E94F922C82F809128
:1012A000F801C81741F1C093F8018091AC0282FFA8
:1012B0001EC080FF04C088E393E00E949E068091D8
:1012C000AC0280FF0CC01F92CF9383E393E09F9307
:1012D0008F930E9437070F900F900F900F9080917F
:1012E000AC0280FF04C081E393E00E949E068C2F35
:1012F000CF910C943B09CF910895CF93DF93CDB755
:10130000DEB72B970FB6F894DEBF0FBECDBF4F836D
:10131000588769877A878B8761110E942B139E01FA
:101320002F5F3F4F86E0F90111928A95E9F785E03A
:10133000FE013796D90101900D928A95E1F78981D6
:101340009A814C815D81452B31F09F3F31F491E0D2
:101350008F3F19F403C091E001C090E090FF09C0F5
:1013600049815A816B817C818D819E810E944912C5
:1013700005C0C9010E94FD078111F2CF2B960FB65F
:10138000F894DEBF0FBECDBFDF91CF910895FC0171
:10139000808191810E94A40F0895CF93882309F43E
:1013A000A9C0C82F8238C1F40E94F92281FDA2C0D1
:1013B00069E380910201909103010E944F240E94F1
:1013C0004D132FEF81EE94E0215080409040E1F7E3
:1013D00000C0000069E319C0833801F50E94F922BA
:1013E00080FD88C063E580910201909103010E9415
:1013F0004F240E944D132FEF81EE94E02150804046
:101400009040E1F700C0000063E5809102019091F7
:1014100003010E945A24CF910C944D138438C1F4D7
:101420000E94F92282FD66C067E4809102019091DA
:1014300003010E944F240E944D132FEF81EE94E090
:10144000215080409040E1F700C0000067E4DDCF0C
:101450008CEF8C0F813AF8F48C2F0E94A22181111D
:1014600049C06C2F80910201909103010E94AD232D
:10147000882349F06C2F80910201909103010E9412
:101480005A240E944D136C2F809102019091030108
:101490000E944F24C0CF80E28C0F883048F4C77080
:1014A00081E001C0880FCA95EAF70E940B13B3CF01
:1014B000EBE5EC0FE33040F4F0E0E95BFE4F8081B8
:1014C00090E0CF910C946B23E8E5EC0FE73150F4FA
:1014D000F0E0EE0FFF1FE75EFE4F80819181CF911C
:1014E0000C948123CD3E30F08C2F0E94F219CF91C5
:1014F0000C94C41ACF910895882309F464C08238EB
:1015000079F40E94F92281FF5EC069E380910201B3
:10151000909103010E944F240E944D1369E310C073
:101520008338B1F40E94F92280FF4DC063E58091B9
:101530000201909103010E944F240E944D1363E524
:1015400080910201909103010E945A240C944D1342
:10155000843879F40E94F92282FF35C067E48091D3
:101560000201909103010E944F240E944D1367E4F1
:10157000E7CF9CEF980F913A10F4682FE1CF90E2FB
:10158000980F983050F4877091E001C0990F8A95B8
:10159000EAF7892F0E941113D9CF9BE5980F93305A
:1015A00020F480E090E00C946B2398E5980F97313D
:1015B00020F480E090E00C9481238D3E20F00E9486
:1015C0004D1A0C94C41A08951F93CF93DF93182FCC
:1015D000EB010E94CD09209741F08FE99FE0019730
:1015E000F1F700C000002197F6CF812FDF91CF9156
:1015F0001F910C947C0A893319F060E070E002C0FE
:1016000060E570E00C94E40A882321F00E940B133B
:101610000C944D130895882321F00E9411130C940B
:101620004D130895CF92DF92EF92FF920F931F9385
:10163000CF93DF937C01D62FC72FFC011281058148
:1016400002950F700E9401138823B9F01123A9F0AD
:101650008C2F807F803421F080E28D0F883068F0FD
:101660008091F80282FD09C082E00E94AD130E94C1
:10167000011391E0D82ED92601C0D12CCC2EC294D2
:101680008FE0C8228C2D90E08C30910508F0CFC1FE
:10169000FC01EA5AFF4F0C942F2D8C2F807FCF70C6
:1016A000882311F0C295C07F112399F0CC2309F44F
:1016B000AAC180E28D0F883010F0D11104C08C2FA8
:1016C0000E940B1303C08C2F0E941E130E944D1307
:1016D0009AC18D2F0E947C0ACC2309F4A8C180E214
:1016E0008D0F883038F1DD2329F18C2F0E942413CF
:1016F00024C08C2F807FCF70803211F0C295C07FC4
:10170000DD2319F0D130A1F13DC08091F80282FFB4
:1017100017C0112349F0CC2329F08C2F0E940B1302
:101720000E944D1380E070C180E00E947C0ACC23AF
:1017300009F47DC18C2F0E9411130E944D1377C1B3
:10174000112371F0002341F0013031F40E942E1377
:101750008C2B0E9436136BC10E942E138C2B1DC044
:10176000002319F0013009F462C10E94431325C01F
:10177000112321F0063008F05AC10EC0053008F0E0
:1017800056C11BC0112361F0002331F0F7018581A0
:1017900080FF39C18F7085838C2F0E94040B47C155
:1017A000002359F0D93309F03FC1FFEF07EE13E0F2
:1017B000F15000401040E1F735C18C2F0E940B0B17
:1017C00036C18C2F86958695837019F0813061F033
:1017D0002EC1112321F08D2F9C2F937002C080E029
:1017E00090E00E946B232BC1112321F08D2F9C2FA1
:1017F000937002C080E090E00E94812320C18D2F71
:10180000112319F00E94F21902C00E944D1A0E9481
:10181000C41A15C18C2F837009F047C011110BC178
:101820002D2F229526952770220F220F6D2F6F7076
:10183000862F90E0A0E0B0E0022E04C0880F991F30
:10184000AA1FBB1F0A94D2F7D4FF10C04FE050E08C
:1018500060E070E004C0440F551F661F771F2A9593
:10186000D2F7409550956095709503C040E050E0E8
:10187000BA01C695C695C3708A019B01082B192B26
:101880002A2B3B2BC901B801C23049F058F4C130B2
:1018900019F00E94210ECFC00E940F0ECCC00E94F2
:1018A000330EC9C00E940D0EC6C0112319F08C2F33
:1018B000817001C08695882309F4BDC02D2F229523
:1018C00026952770220F220F6D2F6F70862F90E0C4
:1018D000A0E0B0E0022E04C0880F991FAA1FBB1F12
:1018E0000A94D2F7D4FF10C04FE050E060E070E0FF
:1018F00004C0440F551F661F771F2A95D2F74095E5
:1019000050956095709503C040E050E0BA01C695CF
:10191000C695C3708A019B01082B192B2A2B3B2BE0
:10192000C901B801C23049F058F4C13019F00E9421
:10193000E60E81C00E94D40E7EC00E94F80E7BC0CD
:101940000E94470E78C0CF70112339F08C2F0E946F
:101950006D0E8D2F0E94040B6EC08D2F0E940B0BFD
:101960008C2F0E948E0E67C0D23F21F128F4D03F09
:1019700041F0D13FC1F043C0D33F19F1D43F79F0DA
:101980003EC0112341F0053008F051C08C2F8F71FB
:101990000E94B30E4CC0063008F049C0F7CF8091CA
:1019A000F80282FF18C0112339F08C2F8F710E942A
:1019B0006D0E3DC01123C9F38C2F8F710E948E0EC6
:1019C00036C0112329F08C2F8F710E94580E2FC022
:1019D0000E94530E2CC0112349F0CF718C2F0E940E
:1019E0006D0E63E08C2F0E94921321C081E00E9453
:1019F000AD130230E0F082E00E94AD1318C0112355
:101A000031F0002391F28D2F0E94CD0910C00023E8
:101A100099F2D93349F41FEF27EE33E011502040FB
:101A20003040E1F700C000008D2F0E947C0A88EF53
:101A30008C0D843020F40E94F9220E943B09DD20A5
:101A4000C9F00E94FD1280FD15C0F70112820E94AC
:101A5000F7120E946D0EC7010E945B0D0E94F712E3
:101A6000DF91CF911F910F91FF90EF90DF90CF907A
:101A70000C948E0EDF91CF911F910F91FF90EF90FC
:101A8000DF90CF9008950F931F93CF93DF93EC01D6
:101A9000688179818A810E94AF0F8C010E940A0FB0
:101AA0000E94FB0DB801CE010E94120BDF91CF9175
:101AB0001F910F910895CF93DF93EC019881898155
:101AC0002B813C81232B31F08F3F31F481E09F3F0C
:101AD00019F403C081E001C080E080FD1DC0CE018B
:101AE0000E941E08811110C00E9401138823A1F0DA
:101AF0008A81882389F08091F80282FD0DC082E0FE
:101B0000DF91CF910C94AD13CE010E94430DCE0115
:101B1000DF91CF910C94FF07DF91CF910895882337
:101B200021F00E941E130C944D130895882321F078
:101B30000E9424130C944D13089580E090E00E94BD
:101B40006B2380E090E00E9481230E942B130E946F
:101B50004D130E94771C0C94C41A8091020190913D
:101B600003010E9465240C949D0D0E941B130C948C
:101B7000AD0D92959F70963079F010F4925001C09F
:101B80009A50923068F4803F69F018F4883E40F42F
:101B900009C0843F29F406C0883E20F0813F11F03F
:101BA00080E0089581E00895FC01808191810E9488
:101BB000A40F0E94B90D0895CF93DF9300D000D0F9
:101BC0001F92CDB7DEB70F900F900F900F900F9030
:101BD000DF91CF910895CF93DF9300D000D000D054
:101BE000CDB7DEB726960FB6F894DEBF0FBECDBFD9
:101BF000DF91CF910895089508950C94FC0D0C94F5
:101C0000FD0D0E94FF0D60931C0270931D028093D6
:101C10001E0290931F020C949D0D0C94010E0F93C5
:101C20001F9300911C0210911D0220911E02309101
:101C30001F02602B712B822B932B1F910F910C9401
:101C4000010E0F931F9300911C0210911D02209111
:101C50001E0230911F0260237123822393231F9160
:101C60000F910C94010E0F931F9300911C02109181
:101C70001D0220911E0230911F02602771278227CA
:101C800093271F910F910C94010E0C94FC0D0E9450
:101C9000450E609318027093190280931A02909374
:101CA0001B020C949D0D60E070E0CB010C94470E7C
:101CB0000F931F9341E050E060E070E08A019B01C8
:101CC00004C0000F111F221F331F8A95D2F7C901CC
:101CD000B8011F910F910C94470E0F931F9341E091
:101CE00050E060E070E004C0440F551F661F771F8E
:101CF0008A95D2F78091180290911902A0911A0248
:101D0000B0911B028A019B01082B192B2A2B3B2B1C
:101D1000C901B8011F910F910C94470E0F931F93A7
:101D200041E050E060E070E004C0440F551F661FC2
:101D3000771F8A95D2F74095509560957095809160
:101D4000180290911902A0911A02B0911B028A0107
:101D50009B01082319232A233B23C901B8011F91A2
:101D60000F910C94470E0F931F9341E050E060E0F9
:101D700070E004C0440F551F661F771F8A95D2F785
:101D80008091180290911902A0911A02B0911B0241
:101D90008A019B01082719272A273B27C901B80177
:101DA0001F910F910C94470E0F931F9300911802EF
:101DB0001091190220911A0230911B02602B712B95
:101DC000822B932B1F910F910C94470E0F931F930F
:101DD000009118021091190220911A0230911B02F1
:101DE00060237123822393231F910F910C94470E3C
:101DF0000F931F93009118021091190220911A025B
:101E000030911B0260277127822793271F910F9122
:101E10000C94470E08952BE0929F800D1124E82F1B
:101E2000E695E695E695877051E001C0550F8A95D5
:101E3000EAF785E0E89FF0011124E650FE4F20E02C
:101E400030E070E04081CB01022E02C0969587956C
:101E50000A94E2F7817081958427852384278193F2
:101E60002F5F3F4F2530310569F708952BE0929F92
:101E7000800D1124682F669566956695982F97704A
:101E800085E0689FB001112440E050E080E0FB0154
:101E9000E40FF51FE650FE4F208130E0092E02C00E
:101EA000369527950A94E2F721703327042E01C056
:101EB000220F0A94EAF7822B4F5F5F4F453051059E
:101EC00031F70895BF92CF92DF92EF92FF920F9376
:101ED0001F93CF93DF938C01C0901802D09019020A
:101EE000E0901A02F0901B0280911C0290911D025A
:101EF000A0911E02B0911F02C82AD92AEA2AFB2A01
:101F0000CFE1D0E0D701C6010C2E04C0B695A7954D
:101F1000979587950A94D2F780FD04C0219790F792
:101F2000B12C07C0BC2EB8018C2F0E94BE160197A1
:101F3000A9F38B2DDF91CF911F910F91FF90EF901F
:101F4000DF90CF90BF900895CF93DF93EC010E9474
:101F5000620FBE010E94BE16DF91CF9108951F93BC
:101F6000CF93DF93EB019091F901992321F0CB01FD
:101F70000E94A40F13C0882349F0CB010E94620F76
:101F8000182F682FCE010E940B0F04C0CB010E94B6
:101F9000360F182FBE01812F0E94BE16DF91CF9100
:101FA0001F9108951F93CF93DF93C091200216E0F5
:101FB00080912102C81799F0D0E01C9FF0011D9F6D
:101FC000F00D1124EE5DFD4F4081518162817381DE
:101FD000848195810E94EB0D2196C770E9CFDF9136
:101FE000CF911F91089540915202509153026091F8
:101FF00054027091550280915602909157020C94B0
:10200000EB0DEF92FF920F931F93CF93DF9380918D
:10201000570282958F7009F065C080915402882321
:1020200009F460C080912002F090210210915202C8
:1020300000915302609155027091560291E01F3F4A
:1020400009F090E0C0910001D0910101292F96E0A4
:10205000E92E8F1509F446C06115710521F00F3F77
:1020600021F030E003C031E001C0322F90E030FDBC
:1020700036C0E89EF001E99EF00D1124DF01AE5D4F
:10208000BD4F11963C911197301329C03C913113EB
:1020900026C012963C911297311121C013964D9192
:1020A0005C911497461B570B4C175D07C0F4809149
:1020B00057028F70806180935702E95DFD4F8081E8
:1020C0008F708061808382E592E00E945B0DDF91DA
:1020D000CF911F910F91FF90EF900C94D20F01962A
:1020E0008770B7CFDF91CF911F910F91FF90EF9045
:1020F00008959F92AF92BF92CF92DF92EF92FF929C
:102100000F931F93CF93DF93CDB7DEB761970FB6D1
:10211000F894DEBF0FBECDBF8C0185E0F801DE0173
:102120001D9601900D928A95E1F7D8011296EC90D8
:1021300090915202E0915302209155023091560243
:102140002115310531F0EF3F31F481E09F3F19F463
:1021500003C081E001C080E0B82FB1709B2E80FDEC
:1021600047C1D8014C9111965C9111971396AD908F
:10217000BC90149782E5C82E82E0D82EF0905402CD
:10218000B501621B730B2091000130910101FF200A
:1021900009F4D9C0809157026217730708F095C0FF
:1021A000282F207F09F052C05E1313C0491311C0BD
:1021B000FE2CE1100EC08F708061809357020E9448
:1021C000F30FC6010E945B0D80915702F8018583D1
:1021D0004DC1AB2831F05F3F31F481E04F3F19F43E
:1021E00003C081E001C080E080FD03C081E08E2556
:1021F00002C080E090E0F82FF170FF2E80FF1CC03D
:10220000809120022091210236E0821709F40BC14F
:1022100090E0389FF001399FF00D1124EE5DFD4FE5
:102220006181561306C06081461303C06281E612C5
:1022300003C001968770E9CFFE2CEE2009F416C189
:102240008091570281608093570254C05E1306C08C
:10225000491304C0E11002C0F80199C0C8010E94EE
:10226000D40D882361F1EE2051F120915702822F85
:1022700082958F7090E0029774F080915202909155
:10228000530298878F831986BB86AA862C87CE0136
:1022900007960E945B0D86E0F801A2E5B2E001908E
:1022A0000D928A95E1F70E9401100E94F30F0AC077
:1022B0005E1711F1C8010E94D40D81112CC0C80114
:1022C0000E945B0DFF24F394D1C0282F207F81F75B
:1022D0007A2DB98AA88A6E2D89890E94DC0D82E543
:1022E00092E00E945B0D86E0D6011D928A95E9F787
:1022F0000E94F30FF12CBAC04913DCCFE110DACF02
:10230000F8018583C8010E945B0D86E0D6011D920D
:102310008A95E9F7ABC0EE2091F220915702822F07
:1023200082958F7090E002970CF4B5CF80915202A5
:10233000909153029A8389831B82BD82AC822E8343
:10234000CE010196A6CF6217730708F044C0FE2C99
:10235000EE2009F4B4CF5E1330C049132EC0209193
:10236000570220FD21C0822F82958F70482F50E0A8
:1023700041155105C9F0F80125834F30510541F051
:102380008F5F982F9295907F822F8F70892B8583F6
:10239000C8010E945B0D86E0F801A2E5B2E0019061
:1023A0000D928A95E1F73CC086E0F801A2E5B2E023
:1023B00001900D928A95E1F759C0C8010E94D40D91
:1023C000811169CF80915702816080935702C801C3
:1023D0000E945B0D4BC07A2DB98AA88A6E2D89891F
:1023E0000E94DC0D86E0D6011D928A95E9F718C09F
:1023F000EE2009F464CFC8010E94D40DF82E882382
:1024000009F45DCF86E0F801A2E5B2E001900D92FB
:102410008A95E1F782E592E00E94C7090E940110C7
:102420000E94F30F23C04D875E878D859E850E9495
:10243000A40F292F22952F70223028F49F7039F095
:10244000811105C00BC0243028F49F7049F4805ED0
:10245000883020F0C8010E945B0D9F2CF92C06C02B
:10246000D80115969C91907F91F7F8CF8F2D6196AA
:102470000FB6F894DEBF0FBECDBFDF91CF911F9195
:102480000F91FF90EF90DF90CF90BF90AF909F9013
:1024900008951F93CF93DF93CDB7DEB72C970FB678
:1024A000F894DEBF0FBECDBF4F83588769877A8708
:1024B0008B879C87CE0107960E9479108823D1F0E4
:1024C0009F8188852A853B85232B31F08F3F31F40E
:1024D00081E09F3F19F403C081E001C080E080FDEE
:1024E00047C04F81588569857A858B859C850E9478
:1024F000EB0D3EC086E0FE013796DE01119601909D
:102500000D928A95E1F7FF81E8856A857B856115E3
:10251000710531F0EF3F31F481E0FF3F19F403C062
:1025200081E001C080E080FD23C02091210230E0E5
:10253000C9010196877099274091200250E08417C5
:102540009507F1F1F983EA837D836C8396E0929F8E
:10255000D001939FB00D1124AE5DBD4FFE013196A9
:1025600001900D929A95E1F7809321020E94D20F7B
:1025700016E08091200290912102891771F1189F35
:10258000C00111248E5D9D4F0E947910882329F18E
:10259000E09120021E9FF0011124EE5DFD4F40816D
:1025A000518162817381848195810E94EB0D8091BC
:1025B000200290E001968770992780932002D9CF5E
:1025C0000E94B50D1092210210922002E2E5F2E085
:1025D00086E0DF011D928A95E9F72C960FB6F894F4
:1025E000DEBF0FBECDBFDF91CF911F9108958091C7
:1025F00078028595859585950895809178028770F4
:10260000089590917802977081E009F480E0089530
:1026100080919B02089590919B02892B80939B024D
:102620000895809590919B02892380939B02089541
:1026300080939B02089510929B02089590919A02B4
:10264000892B80939A020895809590919A0289230C
:1026500080939A02089510929A02089580917902C7
:10266000089508950C9431130C9432139091F8024C
:1026700092FD08C090917902981721F08093790219
:102680000C943413089580917902882329F01092D4
:10269000790280E00C9434130895CF93DF93E09196
:1026A0000201F091030180919B028083E09102017D
:1026B000F0910301908180919A02892B808380910F
:1026C0007902882381F0E0910201F0910301908169
:1026D000892B808380910201909103010E949723AE
:1026E00081110E944313C0910201D091030140E285
:1026F00050E068E572E0CE010E94492D892B69F017
:1027000080E2FE01A8E5B2E001900D928A95E1F722
:10271000CE01DF91CF910C940823DF91CF910895E2
:102720000C9431139091F80292FD10C098E0899FAB
:1027300090011124262B209378020E946D0E809127
:1027400078028595859585950C9490130C946D0E63
:102750001092780280E00C9490132091780280957A
:10276000822380937802982F977099F430E0482F55
:10277000082E000C550B2417350759F09091F802DC
:1027800092FD07C08595859585950E948E0E0C94C7
:10279000A8130895CF939091F80292FB222720F975
:1027A0002817F9F0C82F892FC0FB82F98093F8020F
:1027B0008091F7029091F8020E94261482E00E9414
:1027C000AD138091AC0280FF0CC01F92CF9383E4C5
:1027D00093E09F938F930E9437070F900F900F9075
:1027E0000F90CF9108958091F80282FB882780F99D
:1027F00091E089270C94CA1381E00C94CA1380E0FD
:102800000C94CA1380E090E00E945E2D21E0893E86
:102810009E4F09F020E0822F089582E090E00C9412
:10282000562D83E090E00C94562DCF9384E090E0F9
:102830000E94562DC82F82E290E00E94562D2C2F28
:1028400030E0A901582BCA01CF910895CF93C92F29
:10285000682F84E090E00E94642D6C2F82E290E06B
:10286000CF910C94642DAB01BC018FE090E00C94EF
:10287000762DAB01BC0183E190E00C94762D60E0F5
:1028800070E0CB010C94391460E070E0CB010E9441
:1028900033140C943F1469EE7EEF80E090E00E94C8
:1028A000822D60E082E090E00E94642D60E083E091
:1028B00090E00E94642D10921C0210921D02109252
:1028C0001E0210921F0260E084E090E00E94642DDE
:1028D00060E082E290E00E94642D60E085E090E09C
:1028E0000E94642D60E086E090E00E94642D6FEF0E
:1028F00087E090E00E94642D40E050E0BA0188E05B
:1029000090E00E94762D60E08DE090E00E94642DC2
:1029100040E050E0BA0188E190E00E94762D60E04E
:1029200087E190E00E94642D40E050E0BA018CE124
:1029300090E00E94762D60E070E080E290E00E94DE
:10294000822D40E050E0BA0188E190E00E94762DAF
:102950000C9444140C944B14682F8EE090E00C946B
:10296000642D0E941F256093A8027093A902809392
:10297000AA029093AB026093A4027093A502809385
:10298000A6029093A702089585B7806885BF85B792
:10299000806885BF089581E008950C94CB14089554
:1029A0000C94CF140C94CF140C94D2140C94CF1418
:1029B0000C94D6140C94CF140E94C41489E597E2A9
:1029C0000E94EF220E94DA140C94D8140E94D014B2
:1029D0000C94CF140E949B170E943A090C94AD1CD2
:1029E0000E940A250E94C6180E94EA140C94D4146E
:1029F0005F926F927F928F929F92AF92BF92CF928F
:102A0000DF92EF92FF920F931F93CF93DF93CDB797
:102A1000DEB72A970FB6F894DEBF0FBECDBF0E9477
:102A2000DB18C82E81110E94B1143CE9832E32E0DC
:102A3000932E00E010E0502E802F0E94BF175C0103
:102A4000F401619071904F01682679266114710438
:102A5000B1F40F5F1F4F0430110569F78FEF8983C1
:102A60008A831B820E9413258160782F9D838C832B
:102A700049815A816B818D810E947D093AC0809184
:102A8000AC0281FD0E94C817D12CEE24E394F12CF6
:102A9000C3018E219F21892B29F10E94CD14882307
:102AA000A9F0DE825F82AE20BF2081E0AB2809F46E
:102AB00080E088870E9413258160782F9A87898714
:102AC0004E815F8168858A850E947D09000F111FF4
:102AD000F801E456FD4F80819181E826F926F182C4
:102AE000E08207C0D394EE0CFF1CFBE0DF12D0CFD6
:102AF000B0CF81E0C11001C080E02A960FB6F894F3
:102B0000DEBF0FBECDBFDF91CF911F910F91FF9020
:102B1000EF90DF90CF90BF90AF909F908F907F907D
:102B20006F905F9008950E94F8140E94641B0C94AB
:102B30004B09CF93DF930E94C316EC01811521E569
:102B4000920708F045C0811530E5930708F094C05E
:102B5000883E910528F5803E910508F0F8C0883A36
:102B6000910570F4853A910508F07CC0813091059B
:102B700009F475C008F4E8C0049708F0E8C0E4C0A0
:102B80008F3B910508F0E0C0C85AD0E0CC0FDD1FA4
:102B9000C65BDE4F0990D881C02DCE019464D8C0A9
:102BA000811540E2940758F4811551E0950708F02B
:102BB000CEC08D3E910508F4C7C09065C9C0C1154F
:102BC00080E4D80708F4C0C0DF70CE01906AC0C0AE
:102BD000811525E59207A8F4811534E5930708F0DF
:102BE00095C0811543E5940708F07BC0811552E537
:102BF000950708F061C0D82FCC27CE01816F906A6D
:102C0000A7C0C11589E5D807A0F4C11528E5D207EA
:102C100008F082C0C11536E5D30708F095C08C2FA7
:102C20000E9457178F7190E0D82FCC27CE01906269
:102C30008FC0C1154AE5D40708F474C0CE01905680
:102C40008115904208F080C08D2F8F710E94571718
:102C5000DD27D0628F71AE01582BCA0179C081E0A7
:102C600090E076C0C55AD0E0C858DE4F8881C82FA2
:102C7000D0E0CE0190646CC074E0969587957A950B
:102C8000E1F7282F23703C2F337081E090E002C0E1
:102C9000880F991F3A95E2F79C68AC01522B9A0174
:102CA0009C2F9F709695969550E2959FE001112478
:102CB000C9018C2B9D2B4CC08370992721E030E0FB
:102CC00002C0220F331F8A95E2F79C2F96959695A6
:102CD00080E2989FE0011124C22BD32BCE019C6887
:102CE00037C08370992721E030E002C0220F331FE4
:102CF0008A95E2F79C2F9695969540E2949FE00185
:102D00001124C22BD32BCE019A6822C0D82FCC27F6
:102D1000CE01846F906A1CC0DC2FCC27CE01806F5F
:102D2000906A16C08C2F8F700E94571794E0D6952A
:102D3000C7959A95E1F7CF70D0E0DC2FCC27D0690A
:102D40009E01282BC90104C080E090E001C0CE01A3
:102D5000DF91CF9108952CE2829FC0011124FC01E4
:102D60002BE0729FE00DF11D1124E60FF11DEE0F17
:102D7000FF1FEA5AFE4F8591949108950E94AB1669
:102D80000E94991508958238910569F1B0F4813354
:102D9000910509F46DC048F48932910509F463C0C6
:102DA0008A32910509F469C008958533910509F4C3
:102DB00055C089339105B9F00895833E910569F1B5
:102DC00038F4803E9105B1F0823E910509F10895F5
:102DD000863E9105A9F1873E9105B9F1843E9105A2
:102DE00009F064C023C02091F70220FD4FC021FDEF
:102DF0004DC008958091F70280FD44C08091F80293
:102E000080FF44C08091F70284FD42C083EE4DC034
:102E10008091F70282FF38C0F5CF8091F70282FDE2
:102E200033C08091F80280FD31C0ECCF8091F80270
:102E300081FF32C08091F70284FD2AC087EE35C041
:102E40008091F70283FF26C0F5CF8091F70283FDC2
:102E500021C08091F80281FD1FC0ECCF8091F70264
:102E600085FD1CC01DC08091F70285FD19C016C0EC
:102E70008091F70286FD16C017C08091F70286FD8B
:102E800013C010C089E311C082EE0FC080EE0DC0E8
:102E900080E00BC086EE09C084EE07C089E205C061
:102EA00085E303C08AE201C081E390E00895909138
:102EB000F70292FF0DC0282F2871283019F4877F60
:102EC000846006C0282F2471243011F48B7F886021
:102ED00093FF0DC0282F2871283119F4877E846153
:102EE00006C0282F2471243111F48B7E8861209133
:102EF000F80220FF0DC0382F3871383019F4877F61
:102F0000816006C0382F3171313011F48E7F8860B6
:102F100021FF0DC0282F2871283119F4877E816187
:102F200006C0282F2171213111F48E7E886194FD15
:102F3000877E089508950E940214811102C00E94A4
:102F4000AA140E940D148093AC020E941514909351
:102F5000F8028093F7020E949A170E941114682FBA
:102F600070E080E090E00E940D0E60911802709178
:102F7000190280911A0290911B020C94450EE82FC1
:102F8000F0E0EE0FFF1FEF5FFC4F8081918108950D
:102F9000CF92DF92EF92FF920F931F93CF93DF9325
:102FA00088E693E00E949E0681E0E82E83E0F82EFA
:102FB000C0E0D0E093E6C92E93E0D92E0AE513E0F5
:102FC000DF93CF93DF92CF920E94370780E693E0A2
:102FD0000E949E06F701819191917F010E94200934
:102FE0009F938F931F930F930E94370788E593E079
:102FF0000E949E0621968DB79EB708960FB6F8944C
:103000009EBF0FBE8DBFC430D105D1F6DF91CF91E9
:103010001F910F91FF90EF90DF90CF90089580EA7D
:103020008A95F1F7089500C008950C940F1808953B
:103030000C9417180C9418180C9417180C941C184E
:10304000F894E82FE295EF70F0E031A1282F2F706F
:1030500081E090E001C0880F2A95EAF7982F9095BB
:10306000932391A392A1892B82A3789408950F931F
:103070001F93CF93DF93C6E8D1E089918F3F11F082
:103080000E94201881E0CA38D807B9F7CBE7D1E011
:1030900006E811E089918F3F11F00E9420180C176B
:1030A0001D07C1F7DF91CF911F910F910895BF9236
:1030B000CF92DF92EF92FF920F931F93CF93DF9304
:1030C0008C01C62FD0E0CE018A579E4F6C01FC01C7
:1030D00090819F3F09F450C0B62EF894E92FE295F5
:1030E000EF70F0E081A19F7021E030E001C0220F7D
:1030F0009A95EAF7822B81A382A12095282322A307
:1031000078940E941318EBE7F1E046E851E021E0E3
:1031100030E0E12CF12C61916F3F89F0A62FA29550
:10312000AF70B0E090968C9190E06F7002C0959572
:1031300087956A95E2F780FD02C0C90102C080E070
:1031400090E0E82AF92A220F331F4E175F0719F77C
:10315000F60180818F3F11F00E94201861E0E11498
:10316000F10409F460E08B2D0E941518CC0FDD1FCF
:10317000C00FD11FF982E882DF91CF911F910F918B
:10318000FF90EF90DF90CF90BF9008950E94371886
:1031900088E0E1E0F3E0DF01982F1D929A95E9F7CE
:1031A000E9EFF2E0DF011D928A95E9F784E00E94E1
:1031B00026190C940A08FF920F931F93CF93DF9365
:1031C000CDB7DEB728970FB6F894DEBF0FBECDBFE0
:1031D0008E010F5F1F4F88E0F80111928A95E9F781
:1031E000F12C6F2DC8010E945718F394F4E0FF12E0
:1031F000F8CF48E050E0B80189EF92E00E94492DF5
:10320000FF24F394009709F4F12C892B41F088E016
:10321000F801A9EFB2E001900D928A95E1F72F2D08
:1032200044E061E073E089EF92E00E9427190E9478
:103230000C088F2D28960FB6F894DEBF0FBECDBFB9
:10324000DF91CF911F910F91FF9008950895FF9204
:103250000F931F93CF93DF93F82E092F162FD72F9D
:10326000C42F222349F081E08093AF020E941325EE
:103270009093AE028093AD028091AF028823D9F083
:103280008091AD029091AE020E942B25059798F097
:10329000EF2DF02FA12FBD2F80E090E04C2F50E0BC
:1032A0008417950734F4219131912D933D93019624
:1032B000F7CF1092AF02DF91CF911F910F91FF9046
:1032C00008950E94D5270E94F0140C94E1270E94D3
:1032D000E5270E9493150C9403280E94B1240E94B4
:1032E000BC270E94DC140E9461190E9467190E9489
:1032F000E614FBCF8091B60280FF06C06091090101
:1033000070E0660F771F26C081FF04C0609109013D
:1033100084E005C082FF07C06091090188E0689FD2
:10332000B001112417C09091B5029923D1F060919A
:103330000801961788F72091090188E0289F9001DD
:103340001124929FA001939F500D112470E0CA0197
:103350000E941B2D6038710540F46115710519F448
:1033600006C068E070E0862F08958FE7089581E039
:1033700008958091B60280FF08C06091050170E059
:10338000759567957595679521C081FF06C0609119
:10339000050170E07595679519C082FF04C06091C2
:1033A000050170E010C09091B402992399F06091EA
:1033B00004019617A0F780910501899FC00111248F
:1033C00070E00E941B2D6038710540F46115710595
:1033D00019F406C061E070E0862F08958FE7089524
:1033E00081E008958D3E21F40E947A19819504C0F0
:1033F0008E3E29F40E947A198093BA0208958F3E76
:1034000021F40E947A19819504C0803F29F40E941A
:103410007A198093B9020895893F19F40E94B91965
:1034200005C08A3F31F40E94B91981958093BB028F
:1034300008958B3F21F40E94B919819504C08C3FF7
:1034400029F40E94B9198093BC0208959FE0980F57
:10345000983078F421E030E0A90102C0440F551FF4
:103460009A95E2F7CA019091B802892B8093B8022D
:1034700008958D3F21F48091B60281600BC08E3F8C
:1034800021F48091B602826005C08F3F29F48091BB
:10349000B60284608093B60208958D3E39F490910F
:1034A000BA0297FF35C01092BA0259C08E3E29F475
:1034B0009091BA021916BCF32BC09091B9028F3EBD
:1034C00029F497FF25C01092B90249C0803F19F432
:1034D0001916CCF31DC09091BB02893F29F419162F
:1034E000BCF41092BB023BC08A3F19F497FF10C096
:1034F000F8CF8B3F39F49091BC0297FF09C010922E
:10350000BC022DC08C3F21F49091BC021916BCF373
:103510009FE0980F983080F421E030E0A90102C0CC
:10352000440F551F9A95E2F7CA0180959091B80211
:1035300089238093B80213C08D3F21F48091B60295
:103540008E7F0BC08E3F21F48091B6028D7F05C027
:103550008F3F29F48091B6028B7F8093B6028091D1
:10356000B902811106C08091BA02811102C0109285
:10357000B5028091BB02811106C08091BC0281110D
:1035800002C01092B40208958091AC0283FF7EC005
:1035900086EA93E00E949E068091B8021F928F9364
:1035A00081EA93E09F938F930E9437078FE993E01E
:1035B0000E949E068091B902282F082E000C330B22
:1035C0003F938F938CE993E09F938F930E943707EB
:1035D0008AE993E00E949E068091BA02282F082E65
:1035E000000C330B3F938F9387E993E09F938F9366
:1035F0000E94370785E993E00E949E068091BB02F6
:10360000282F082E000C330B3F938F9382E993E011
:103610009F938F930E94370780E993E00E949E0654
:103620008091BC02282F082E000C330B3F938F9300
:103630008DE893E09F938F930E9437078AE893E089
:103640000E949E068091B5021F928F9387E893E0B7
:103650009F938F930E94370785E893E00E949E0610
:103660008091B6021F928F9382E893E09F938F938D
:103670000E9437078FE793E00E949E068DB79EB7A2
:103680004C960FB6F8949EBF0FBE8DBF0E941325B7
:103690002091B902211104C02091BA02222321F005
:1036A0009093B3028093B2022091BB02211104C017
:1036B0002091BC02222321F09093B1028093B002AA
:1036C00087EB92E00C945D23EF92FF920F931F9390
:1036D000CF93DF9300D000D000D0CDB7DEB786E027
:1036E000E7EBF2E0DE01119601900D928A95E1F789
:1036F000E090B902F090BA020091BB021091BC02B6
:103700001092B9021092BA021092BB021092BC023F
:10371000E11003C0FF2009F45DC08091B2029091D6
:10372000B3020E942B25AC019091B502992339F088
:1037300020910A0130E02417350758F04BC0209142
:103740000B018AE0289F900111242417350718F0F7
:1037500041C09F3F19F09F5F9093B502EE2061F04A
:103760000E947A191E1414F09FEF01C091E0989FF7
:10377000902D11249093B902FF2061F00E947A19D4
:103780001F1414F09FEF01C091E0989F902D112419
:103790009093BA023091B9023323E1F02091BA023A
:1037A0002223C1F045EB3403C0011124992319F001
:1037B0009093B90203C081E08093B90235EB2303F3
:1037C000C0011124992319F09093BA0203C081E03B
:1037D0008093BA02011103C0112309F45DC08091E6
:1037E000B0029091B1020E942B25AC019091B402DD
:1037F000992339F02091060130E02417350758F05D
:103800004BC0209107018AE0289F900111242417C2
:10381000350718F041C09F3F19F09F5F9093B402A5
:10382000002361F00E94B919101614F09FEF01C037
:1038300091E0989F902D11249093BB02112361F089
:103840000E94B919111614F09FEF01C091E0989FE2
:10385000902D11249093BC023091BB023323E1F0F0
:103860002091BC022223C1F045EB3403C001112496
:10387000992319F09093BB0203C081E08093BB02AF
:1038800035EB2303C0011124992319F09093BC0256
:1038900003C081E08093BC028091B90281110BC00A
:1038A0008091BA02811107C08091BB02811103C0CF
:1038B0008091BC0281110E94C41AEB82FC820D83AC
:1038C0001E8386E0FE013196A7EBB2E001900D92D7
:1038D0008A95E1F726960FB6F894DEBF0FBECDBFEE
:1038E000DF91CF911F910F91FF90EF900895E7EB3B
:1038F000F2E086E0DF011D928A95E9F71092B502A9
:103900001092B4021092B6020895CF93DF9397FFFE
:103910000DC0FB012281222349F0EC010E94EC1C26
:10392000CE019F770E945F1D0E94391D81E0DF91CB
:10393000CF91089590910A03923069F48A3040F44F
:1039400090E009966AE070E00E941B2D875A01C042
:1039500086500C94FB0A0C9404098CE090E00E94C1
:10396000562D90E0A0E0B0E080930A0390930B0303
:10397000A0930C03B0930D038091AC0280FF0EC0A6
:1039800080910A031F928F9388EE93E09F938F9309
:103990000E9437070F900F900F900F90089560913D
:1039A0000A038CE090E00C94642D80930A030E943B
:1039B000CF1C8091AC0280FF0EC080910A031F9241
:1039C0008F9389EC93E09F938F930E9437070F901A
:1039D0000F900F900F9008950E9405238695817097
:1039E00080930F030E9405238170809309038091C7
:1039F0000A03813039F480910F03882319F089E399
:103A00000E94FB0A0E94081380930E030E941B135E
:103A100080910A03813071F048F0823081F0843067
:103A200009F586EE0E94FB0A88E11AC082EE0E9428
:103A3000CD0918C088E193E00E94A20713C08091CD
:103A40000903811103C083E50E94FB0A82EE0E94F4
:103A5000CD098FE39CE90197F1F700C0000087E5ED
:103A60000E94FB0A8FE39CE90197F1F700C0000078
:103A7000089580910A03813059F030F0823089F046
:103A80008430C9F488E215C082EE0E947C0A13C01B
:103A90008CE20E94FB0A80910F03882361F089E386
:103AA00008C082EE0E947C0A80910903811103C044
:103AB00083E50E94FB0A80910E030C9418130F9368
:103AC0001F93CF93DF938C01CCE0D0E0C8010C2E84
:103AD00002C0969587950A94E2F78F700E949A1C0F
:103AE0002497CC3F8FEFD80789F7DF91CF911F91B3
:103AF0000F9108950F931F93CF93DF93EC018B01E8
:103B0000FB018281882351F00E940813CE01825E5E
:103B10009C458530910510F40E94D51CB801CE015A
:103B2000DF91CF911F910F910C94851CCF93DF9360
:103B3000EC01FB018281882309F43CC1C430FDE51E
:103B4000DF0760F4CB3F9CE5D90788F49E01225043
:103B50003C452431310508F02EC109C0C236EDE5DF
:103B6000DE0729F0C63AFDE5DF0709F024C10E940F
:103B700015149093F8028093F702C1318CE5D807B1
:103B800009F4C6C008F042C0C930ECE5DE0709F40C
:103B90009BC000F5C5308CE5D80709F485C078F4E2
:103BA000C330ECE5DE0709F478C008F07AC0C23013
:103BB000DC4509F0F5C08091F7028160EFC0C730A5
:103BC0009CE5D90709F478C008F07AC08091F70223
:103BD0008061E4C0CD30FCE5DF0709F487C058F40C
:103BE000CB309CE5D90709F479C008F07BC08091FF
:103BF000F70288606FC0CF30FCE5DF0709F480C0B2
:103C000008F082C08091F702877FC8C0CE3F9CE554
:103C1000D90709F471C000F5C531FCE5DF0709F4E7
:103C200085C068F4C3319CE5D90709F475C008F074
:103C300095C00E94B50D8091F7028F77AFC0CC3F41
:103C4000FCE5DF07A9F108F054C0CB3FDC4509F0E3
:103C5000A7C08091F80240C0C230EDE5DE0709F44C
:103C600089C058F4C1158DE5D80709F45AC008F089
:103C700069C08091F80282602FC0C236EDE5DE0790
:103C800009F47CC0C63AFDE5DF0709F481C0C33002
:103C9000DD4509F085C080E06EC08091F70282604A
:103CA0007DC08091F70216C08091F702886076C0CF
:103CB0008091F80282604FC08091F70280626EC0EE
:103CC0008091F70280646AC00E94B50D8091F7026E
:103CD000806864C0846062C081603DC08091F702EA
:103CE0008E7F5CC08091F7028D7F58C08091F70273
:103CF00016C08091F80218C08091F8028D7F2BC009
:103D00008091F7028F7E4AC08091F7028F7D46C076
:103D10008091F7028F7B42C08091F702877F8B7F73
:103D20003DC08091F8028D7F8E7F15C08091F70293
:103D300082FB222720F991E0922790FB82F990FBE9
:103D400083F92CC08091F802982F909591708E7F06
:103D5000892B90FB81F98093F80222C00E94B50D57
:103D60008091F70287FB222720F991E0922790FBB0
:103D700087F914C081E00E94AC1412C08091F70250
:103D800084FB222720F991E0922790FB84F906C05A
:103D90008091F702982F909590FB80F98093F7021D
:103DA0008091F7029091F8020E9426140E94B50DAE
:103DB00080E001C081E0DF91CF91089580910401FE
:103DC0001F928F93809105011F928F93809108011C
:103DD0001F928F93809109011F928F9380910A0106
:103DE0001F928F9380910B011F928F9388E094E034
:103DF0009F938F930E9437078DB79EB70E960FB68D
:103E0000F8949EBF0FBE8DBF0895883220F58E3185
:103E100008F068C08B3091F1C0F4873009F0BEC063
:103E200081E080930B0184E180930A018AE0809312
:103E300009018EE18093080188E08093050188E202
:103E4000809304018AE695E0C6C0833109F443C03B
:103E5000843169F1A3C08F3409F49EC028F48932FB
:103E600031F1883359F09AC0813531F008F4D4C06B
:103E7000823509F4A7C092C08FEFA5C08CE895E009
:103E80000E949E060E94DE1E1F9281E08F931F9269
:103E900088E08F9385E894E09F938F930E94370783
:103EA0000F900F900F900F900F900F9096C089E891
:103EB00095E00E949E068091C102882309F4AAC061
:103EC0001092C1021092C0021092BF021092BE0264
:103ED0001092BD02B1C08BE795E00E949E060E9441
:103EE000DE1E7BC08D518093C102833031F170F4AE
:103EF0008130D1F0823009F03FC08AE091E09093A8
:103F0000C0028093BF0287E991E01FC0853059F15C
:103F100008F1863089F584E091E09093C0028093A7
:103F2000BF0282ED91E011C08BE091E09093C0025E
:103F30008093BF028EE891E008C089E091E0909301
:103F4000C0028093BF0283EA91E09093BE02809307
:103F5000BD0218C088E091E09093C0028093BF0238
:103F600080EB91E0F2CF85E091E09093C0028093E6
:103F7000BF028FEB91E0E9CF1092C10288E795E094
:103F80000E949E068091C102882309F455C01F92A9
:103F90008F9384E795E00DC08AE015C087E695E031
:103FA0001AC097FF47C0108280811F928F9381E6CD
:103FB00095E09F938F930E9437070F900F900F907B
:103FC0000F900BC081E0E091BF02F091C0023097EA
:103FD00029F58EE595E00E949E062091C1022223DC
:103FE00059F18091BD029091BE02009711F48AE8C8
:103FF00091E09F938F931F922F9385E595E09F9378
:104000008F930E9437070F900F900F900F900F9093
:104010000F9016C080E0089586EFD5CF2081082E3E
:10402000000C990B820F911D8F3F910509F00CF444
:10403000B8CF8FEF8083B8CF81E595E00E949E06D0
:1040400081E00895CF93C82F1F928F9382EA95E065
:104050009F938F930E94370781E090E0A0E0B0E04B
:10406000BC01CD0104C0660F771F881F991FCA9538
:10407000D2F70E940D0E0F900F900F900F90CF91DE
:104080000C94B50DDF92EF92FF920F931F93CF9395
:10409000DF93482F50E0FA013597EF33F10508F030
:1040A0003FC1EE59FF4F0C942F2D0E9411141F9207
:1040B0008F9384EF99E09F938F930E9437070E941C
:1040C0000D1483FB992790F91F929F9382FB9927E8
:1040D00090F91F929F9381FB992790F91F929F93CC
:1040E000982F91701F929F931F928F938BEA99E064
:1040F0009F938F930E9437070E94151487FB2227F6
:1041000020F91F922F9386FB222720F91F922F93CD
:1041100085FB222720F91F922F9384FB222720F969
:104120001F922F9383FB222720F91F922F9382FB4C
:10413000222720F91F922F9391FB222720F91F920B
:104140002F93292F21701F922F9381FB222720F973
:104150001F922F93282F21701F922F939F938F933D
:1041600086EC98E09F938F930E9437078DB79EB798
:1041700088960FB6F8949EBF0FBE8DBF06C084EB25
:104180009AE00E949E060E94AA14C1E0CEC084E17B
:1041900097E074C08091AC02817F8E7F8093AC02E7
:1041A0008DEE96E00E949E0680EB9AE00E949E06AD
:1041B00081E08093C202E9CF84E99AE00E949E06E2
:1041C0000E940F08E2CF8091AC02C82FC095C17049
:1041D000C0FB80F98093AC02CC2319F088E89AE008
:1041E00091C08BE79AE00E949E068091AC02897F85
:1041F000877F8093AC02C9CF9091AC0291FBCC2712
:10420000C0F981E0C827892FC0FB81F98093AC02F7
:10421000CC2319F08EE69AE027C080E69AE02EC003
:104220009091AC0292FBCC27C0F981E0C827892F7E
:10423000C0FB82F98093AC02CC2319F081E59AE0AF
:1042400013C081E49AE01AC09091AC0293FBCC2792
:10425000C0F981E0C827892FC0FB83F98093AC02A5
:10426000CC2351F085E39AE00E949E068091AC0237
:1042700081608093AC0259C088E29AE00E949E0659
:1042800084CF8BE296E0FACF0E941F25062FF72EEF
:10429000E82ED92EC091F702C7FBCC27C0F91091A8
:1042A000F602D09118010E94F922DF92EF92FF925C
:1042B0000F931F92CF931F921F931F92DF931F9212
:1042C0008F9387EA95E09F938F930E9437078DB76E
:1042D0009EB70E960FB6F8949EBF0FBE8DBF55CFFA
:1042E0000E94B50D9091F70297FBCC27C0F981E0B1
:1042F000C827892FC0FB87F98093F702CC2329F0C8
:104300008EE19AE00E949E0610C083E19AE0B6CF4B
:10431000895303C08D5101C080E00E94222035CF17
:1043200081E19AE00E949E06C0E08C2FDF91CF9140
:104330001F910F91FF90EF90DF90089580E0089516
:104340000C949E21CF93C82F8091C202813071F0CE
:1043500040F0823009F045C08C2F0E94051F81E09B
:1043600046C00E9408138232F1F504C00E9408136F
:10437000823261F48C2F0E94A021811104C08C2F05
:104380000E9442202CC081E090E029C08C2F0E9426
:104390009E21811123C0C431C9F058F4CB3069F09B
:1043A000C031B9F482E08093C20288E30E94051F05
:1043B00015C0C93259F0C83361F48DEE96E00E9401
:1043C0009E068EE995E00E949E0608C01092C202E9
:1043D0000CC08CE995E00E949E0607C081E08170C8
:1043E00006C01092C20280E002C080E0F8CFCF91F8
:1043F0000895CF93DF9386319C4541F5EB010E94F0
:104400000813982F8A81209102013091030188239B
:1044100079F09A7A81E009F480E08093C3029111E7
:1044200002C069E201C065E3C9010E944F240AC0CD
:104430008091C302811102C069E201C065E3C90134
:104440000E945A240E944D1380E001C081E0DF9158
:10445000CF9108950F931F93CF93DF93C42FD22F43
:10446000FC0182818823C9F04093C6020E94132573
:104470009093C5028093C40280E28C0F883008F0CC
:1044800057C0C77081E001C0880FCA95EAF7DF9175
:10449000CF911F910F910C94040B8091C602481389
:1044A00030C08091C4029091C5020E942B25883CA7
:1044B000910538F510E21D0FCD17B9F080E28C0F91
:1044C000883040F4C77081E001C0880FCA95EAF7D0
:1044D0000E940B0B183028F581E09D2F977001C0CA
:1044E000880F9A95EAF70E94040B802F0E94FB0A1E
:1044F0001830F0F4D77081E001C0880FDA95EAF740
:104500000AC080E28C0F883098F4C77081E001C047
:10451000880FCA95EAF7DF91CF911F910F910C9404
:104520000B0B802FDF91CF911F910F910C94FB0A01
:10453000DF91CF911F910F9108950F939C01CB01B3
:10454000243F4CE5340731F188F4293DFCE53F0771
:10455000D9F02A3D4CE5340779F1283D3C45A9F5D1
:1045600006E221EE41EE68ED7CE52BC0263FFCE53E
:104570003F07E1F0A8F0273F3C4539F507E225EE7B
:1045800046EE67EF7CE51DC007E225EE45EE69EDDE
:104590007CE517C006E221EE40EE64EF7CE511C039
:1045A00007E225EE44EE65EF7CE50BC006E221EE66
:1045B00042EE66EF7CE505C008E221E045EE6AEDDB
:1045C0007CE50E942A2280E008C0FC0182818823C9
:1045D00019F01092C60201C081E00F9108959093E6
:1045E000F7018093F60108959093CC028093CB025B
:1045F0000895E091CB02F091CC02309721F0019028
:10460000F081E02D099480E008950E94F922089538
:10461000EF92FF921F93CF93DF93FC01A091CB0207
:10462000B091CC02109709F442C080911801882300
:1046300041F08091F70287FF04C08081818386E08A
:104640008083EF011296ED91FC911397CE010995AD
:104650008091AC0282FF2BC080FF04C08DEC9AE0F9
:104660000E949E0618E087ECE82E8AE0F82E8091E2
:10467000AC0280FF0BC088811F928F93FF92EF9254
:104680000E9437070F900F900F900F9011502196B6
:104690001111EDCF8091AC0280FF09C085EC9AE04A
:1046A000DF91CF911F91FF90EF900C949E06DF91C8
:1046B000CF911F91FF90EF900895E091CB02F09180
:1046C000CC02309739F022E0DC012C930480F58194
:1046D000E02D099408952091C9023091CA0228174B
:1046E000390771F09093CA028093C902E091CB021E
:1046F000F091CC02309721F00680F781E02D0994EB
:1047000008952091C7023091C8022817390771F027
:104710009093C8028093C702E091CB02F091CC0243
:10472000309721F00084F185E02D09940895FC0173
:10473000329680911801882331F08091F70287FF2B
:1047400002C09EE101C096E080E0915028F02191E6
:104750002223D9F38F5FF9CF0895662351F1209179
:1047600018012223E9F02091F70227FF19C0462FF4
:104770004695469546954E31E0F4677021E030E06D
:1047800002C0220F331F6A95E2F7FC01E40FF11D0E
:10479000828190E02823392381E0232B69F409C02A
:1047A000FC01329608962191621729F0E817F90763
:1047B000D1F780E0089581E008959C01FC013296D4
:1047C0009FEF80E04191461789F09F3F19F4411116
:1047D00001C0982F8F5F8630A9F79F3F39F0F9010C
:1047E000E90FF11D97FDFA956283089508959C01E4
:1047F0002A5F3F4FFC014281461301C0128201969D
:1048000082179307B9F70895262F269526952695A2
:104810002E3170F4FC01E20FF11D677021E030E0F1
:1048200001C0220F6A95EAF78281282B228308951E
:104830008091AC0280FF0CC01F926F938DEF9AE0C5
:104840009F938F930E9437070F900F900F900F90B8
:104850000895262F2695269526952E3178F4FC016D
:10486000E20FF11D677021E030E001C0220F6A9570
:10487000EAF7209582812823228308958091AC0253
:1048800080FF0CC01F926F938FED9AE09F938F93E0
:104890000E9437070F900F900F900F90089520916E
:1048A0001801222329F02091F70227FD0C940424FB
:1048B0000C94DD2320911801222329F02091F70286
:1048C00027FD0C9429240C94F72320911801FC0156
:1048D0003296222331F08091F70287FF02C08EE1E9
:1048E00001C086E0DF011D928A95E9F708950895D9
:1048F0000C94772483E08093CD020C94782481116A
:1049000002C081E001C082E08093CD020C94782443
:104910000C947F2481E08093CD020C9478240C9435
:104920008A2408950C9491240C9492240C9491243C
:104930000C9491240C949124CF930E9498240E946B
:10494000DB180E949624C0E08C2F0E94BF17892B91
:1049500029F4CF5FC430C1F780E001C081E0CF917E
:10496000089508951F920F920FB60F9211248F93FE
:104970009F93AF93BF938091CE02811113C080911A
:10498000100390911103A0911203B091130341966B
:10499000A11DB11D8093100390931103A0931203E6
:1049A000B0931303BF91AF919F918F910F900FBE62
:1049B0000F901F90189580911803843031F10E9458
:1049C00096081092CE0220E488E190E00FB6F894A9
:1049D000A895809360000FBE2093600083B7817F0D
:1049E000846083BF83B7816083BF7894889583B7E1
:1049F0008E7F83BF0FB6F894A89580916000886180
:104A000080936000109260000FBE08950E94B50D63
:104A10000C949A0882E084BD93E095BD9AEF97BD0F
:104A200080936E0008952FB7F894809110039091B1
:104A30001103A0911203B09113032FBF08952FB754
:104A4000F89460911003709111038091120390917A
:104A500013032FBF08959C014FB7F8948091100362
:104A600090911103A0911203B09113034FBF821BC9
:104A7000930B089578941F920F920FB60F92112402
:104A80008F939F93AF93BF938091100390911103E5
:104A9000A0911203B09113030196A11DB11D809343
:104AA000100390931103A0931203B0931303BF91CB
:104AB000AF919F918F910F900FBE0F901F901895FF
:104AC00087E797E790930108809300089AE088E1D0
:104AD0000FB6F894A895809360000FBE9093600085
:104AE000FFCF8091F5020895089522E02093E90018
:104AF0002FEF3091E800215035FD06C035ED3A9595
:104B0000F1F700002111F5CF2091E80025FF0BC03F
:104B100040E050E066E070E00E9472288091E8007A
:104B20008E778093E8000895CF93DF93209118014A
:104B3000222339F02091F70227FF03C060E222E030
:104B400002C068E021E02093E9002FEF3091E800F7
:104B5000215035FD06C035ED3A95F1F700002111E1
:104B6000F5CF2091E80025FF1DC0EC0180911801D0
:104B7000811105C040E050E068E070E003C070E0E3
:104B800040E050E0CE010E9472288091E8008E77CC
:104B90008093E80080E2FE01A5EDB2E001900D9265
:104BA0008A95E1F7DF91CF9108958093D1027093B8
:104BB000D3026093D20280911803843001F582E021
:104BC0008093E9008FEF9091E800815095FD06C039
:104BD00095ED9A95F1F700008111F5CF8091E800ED
:104BE00085FF0DC040E050E063E070E081ED92E0B1
:104BF0000E9472288091E8008E778093E8000895E3
:104C0000BC0184E00C94D525BC0183E00C94D5252F
:104C10008FE29BE00E949E0680911703811109C0DC
:104C20000E94032A0E94602A8091E200846080939F
:104C3000E20008958BE29BE00E949E06109217030B
:104C4000089587E29BE00E949E060C948F2483E2E5
:104C50009BE00E949E066091140381E0611101C0F7
:104C600080E00C947A248FE19BE00E949E06909154
:104C7000180381E0943009F080E0609114030C94F3
:104C80007F242091D0022F5F822F62E30E940F2D9C
:104C9000992319F02093D00208951092D0028091A8
:104CA000D402882371F180911803843041F58091FA
:104CB000E9008F702091EC00922F917020FD90E818
:104CC000892B93E09093E9009091EB0090FF14C042
:104CD0009091EE0097FF10C09091E80095FF03C0FF
:104CE0001092F100F9CF9091E80090FF05C09091EB
:104CF000E8009E779093E8008F708093E90010920F
:104D0000D402089542E061EC81E00E947C2942E2F5
:104D100061EC82E00E947C2942E261EC83E00E9427
:104D20007C299091180381E0943009F080E0609133
:104D300014030C94882480911A03833009F461C011
:104D400030F4813071F0823009F49AC008958A30CD
:104D500009F486C08B3009F46CC0893009F0A8C012
:104D600020C080911903813A09F0A2C08091E80027
:104D7000877F8093E80080911D0390911E03892B0B
:104D800021F460E285ED92E003C060E080E090E015
:104D900070E00E94BD288091E8008B778093E80046
:104DA000089580911903813209F082C080911D031A
:104DB00090911E03029708F07BC08091E800877FE6
:104DC0008093E8008091E80082FD05C0809118037F
:104DD0008111F8CF6DC02091F3008091F20090E036
:104DE000922B029731F48091F100813011F08630DE
:104DF00021F48091F1008093F5028091E8008B7797
:104E000053C080911903813A09F052C080911D036B
:104E100090911E03892B09F04BC08091E800877F99
:104E20008093E8008091E80080FFFCCF809118011A
:104E300036C0809119038132D9F580911D0390917C
:104E40001E03892BA9F58091E800877F8093E800F5
:104E50000E94B12980911B03809318010C94B50D19
:104E600080911903813221F58091E800877F80933A
:104E7000E8000E94B12980911C038093F6020895F6
:104E800080911903813AA1F48091E800877F809393
:104E9000E8008091E80080FFFCCF8091F6028093CB
:104EA000F1008091E8008E778093E8000C94B1299E
:104EB00008959FB7F8941092D4029FBF9091180361
:104EC000943009F057C09091E9009F703091EC0048
:104ED000232F217030FD20E8922B23E02093E9005E
:104EE0002091EB0020FF43C02091EE0027FF3FC040
:104EF0002091CF02222321F02091E80025FF37C026
:104F00001092CF0226E03091E80035FD15C03091B7
:104F10001803343061F53091EB0035FD28C0215085
:104F200021F481E08093CF0222C0EFE9FFE03197C6
:104F3000F1F700C00000E7CF8093F1008091E80016
:104F400085FD0AC08091E80080FFFCCF8091E800D9
:104F50008E778093E80006C08FB7F89421E0209305
:104F6000D4028FBF9F709093E90080E008959F70F6
:104F70009093E9008FEF089584B7877F84BF0FB6C1
:104F8000F894A895809160008861809360001092E9
:104F900060000FBE90E080E80FB6F8948093610047
:104FA000909361000FBE0C948A240E94032A0E94F1
:104FB000602AE2EEF0E080818460808378940C9433
:104FC000F42C8CE091E00C94F4228091180385304D
:104FD000C9F48BE19BE00E949E0680911803853006
:104FE00079F40E94DB24809116038823B1F30E9498
:104FF0009C24882391F30E945C280E94B50DEDCF7C
:105000000C940625089508950C940628292F33271B
:1050100023303105C9F060F42130310581F02230B0
:10502000310509F041C08BE590E021E63BE040C04E
:1050300021323105E1F02232310531F135C082E112
:1050400090E02CEB3BE034C099278130910549F08A
:1050500028F0029749F5E3E3FBE005C0EDE5FBE04E
:1050600002C0E3E4FBE0849190E09F0121C0633043
:105070007105D0F4660F771FFB01E051FE4F2081D0
:10508000318189E090E014C06330710568F4FB0160
:10509000EE0FFF1FE651FE4F20813181FB01E951E8
:1050A000FE4F808190E004C080E090E020E030E09E
:1050B000FA0131832083089580E189BD82E189BDB1
:1050C00009B400FEFDCF8091D8008F7D8093D80079
:1050D0008091E00082608093E0008091E00081FD9B
:1050E000FCCF0895CF92DF92EF92FF920F931F9320
:1050F000CF93DF93EC018B017A010E94D0298111BB
:1051000033C0E114F10439F0F70180819181081B6B
:10511000190BC80FD91FC12CD12C0115110519F17C
:105120008091E80085FD16C08091E8008E7780931D
:10513000E800E114F10449F0F70180819181C80E83
:10514000D91ED182C08285E00FC00E94D029882359
:1051500021F30AC089918093F10001501109FFEFFA
:10516000CF1ADF0ADACF80E0DF91CF911F910F9144
:10517000FF90EF90DF90CF90089520911F03309122
:1051800020032617370748F06115710539F420917F
:10519000E8002E772093E80001C0B901FC0120E06F
:1051A0006115710579F1809118038823F1F185303B
:1051B000F1F18091E80083FD3CC08091E80082FD20
:1051C0002EC08091E80080FFEBCF2091F30080910A
:1051D000F20090E0922B6115710551F08830910535
:1051E00038F421912093F100615071090196F3CFB9
:1051F00021E0089709F020E08091E8008E77809305
:10520000E800CECF2111CFCF0AC0809118038823A8
:1052100061F0853061F08091E80083FD0AC08091E3
:10522000E80082FFF2CF80E0089582E0089583E0F5
:10523000089581E0089520911F03309120032617DF
:10524000370748F06115710539F42091E8002E7791
:105250002093E80001C0B901FC0120E0611571054F
:1052600091F180911803882309F440C0853009F436
:105270003FC08091E80083FD3DC08091E80082FD41
:105280002FC08091E80080FFE9CF2091F30080914A
:10529000F20090E0922B6115710559F0883091056C
:1052A00040F424912093F1003196615071090196E8
:1052B000F2CF21E0089709F020E08091E8008E7796
:1052C0008093E800CBCF2111CCCF0AC08091180386
:1052D000882361F0853061F08091E80083FD0AC089
:1052E0008091E80082FFF2CF80E0089582E0089587
:1052F00083E0089581E00895982F973068F59093A2
:10530000E900981739F07091EC002091ED00509170
:10531000F00003C0242F762F50E021FD02C09F5FD4
:10532000ECCF3091EB003E7F3093EB003091ED00FD
:105330003D7F3093ED003091EB0031603093EB0016
:105340007093EC002093ED005093F0002091EE005C
:1053500027FDE5CF80E008958F708093E90081E01C
:1053600008958091190387FF11C08091E80082FDA4
:1053700005C0809118038111F8CF11C08091E80019
:105380008B770BC080911803882349F08091E80047
:1053900080FFF8CF8091E8008E778093E800089531
:1053A0002091E4003091E50095E64091EC00842FD7
:1053B000817040FF23C08091E80080FD1DC0809176
:1053C0001803882399F0853099F08091EB0085FDD2
:1053D00011C04091E4005091E5002417350729F3EE
:1053E000915011F09A01E1CF84E0089582E0089590
:1053F00083E0089581E0089580E008954091E800F9
:1054000042FFDDCF08950E94712A0E94792AE0EEC2
:10541000F0E0808181608083E8EDF0E080818F772B
:10542000808319BCA7EDB0E08C918E7F8C93808136
:105430008F7E80831092170308950F931F93CF934D
:10544000DF930E94712A0E94792AC8EDD0E08881FA
:105450008F77888388818068888388818F7D88831F
:1054600019BC109218031092140310921603109294
:10547000150300EE10E0F80180818B7F8083888126
:105480008160888342E060E080E00E947C29E1EE58
:10549000F0E080818E7F8083E2EEF0E080818160A9
:1054A0008083808188608083F80180818E7F808303
:1054B000888180618883DF91CF911F910F9108953A
:1054C000E8EDF0E080818F7E8083E7EDF0E0808181
:1054D0008160808384E082BF81E0809317030C9415
:1054E0001D2AE8EDF0E080818E7F80831092E2003B
:1054F00008951092DA001092E10008951F920F9221
:105500000FB60F9211242F933F934F935F936F9396
:105510007F938F939F93AF93BF93EF93FF9380916C
:10552000E10082FF0BC08091E20082FF07C0809102
:10553000E1008B7F8093E1000E9441268091DA0098
:1055400080FF1FC08091D80080FF1BC08091DA00CF
:105550008E7F8093DA008091D90080FF0DC080E1BA
:1055600089BD82E189BD09B400FEFDCF81E0809351
:1055700018030E94082605C019BC109218030E9447
:105580001A268091E10080FF19C08091E20080FF1F
:1055900015C08091E2008E7F8093E2008091E2004E
:1055A00080618093E2008091D80080628093D8006F
:1055B00019BC85E0809318030E9427268091E100A2
:1055C00084FF30C08091E20084FF2CC080E189BD5F
:1055D00082E189BD09B400FEFDCF8091D8008F7DA6
:1055E0008093D8008091E1008F7E8093E1008091CC
:1055F000E2008F7E8093E2008091E20081608093E0
:10560000E20080911403882311F084E007C08091A8
:10561000E30087FD02C081E001C083E080931803AE
:105620000E9433268091E10083FF29C08091E2002F
:1056300083FF25C08091E100877F8093E10082E0B5
:1056400080931803109214038091E1008E7F809361
:10565000E1008091E2008E7F8093E2008091E20081
:1056600080618093E20042E060E080E00E947C295B
:105670008091F00088608093F0000E942126FF91C5
:10568000EF91BF91AF919F918F917F916F915F91BA
:105690004F913F912F910F900FBE0F901F90189533
:1056A0001F920F920FB60F9211242F933F934F9397
:1056B0005F936F937F938F939F93AF93BF93CF939A
:1056C000DF93EF93FF93C091E900CF708091EC00DE
:1056D000D82FD17080FDD0E81092E9008091F000C1
:1056E000877F8093F00078940E94942B1092E900B9
:1056F0008091F00088608093F000CD2BCF70C09334
:10570000E900FF91EF91DF91CF91BF91AF919F9110
:105710008F917F916F915F914F913F912F910F905A
:105720000FBE0F901F9018951F93CF93DF93CDB7A7
:10573000DEB7AA970FB6F894DEBF0FBECDBFE9E182
:10574000F3E08091F100819323E0E132F207C9F7A1
:105750000E949B268091E80083FF2EC1809119034F
:1057600090911A03492F50E04A30510508F024C1A6
:10577000FA01EF55FF4F0C942F2D803821F082381D
:1057800009F01AC108C0809115039091160399235E
:1057900089F082600FC080911D038F70873008F000
:1057A0000BC18093E9008091EB0085FB882780F98D
:1057B0001092E9009091E800977F9093E800809321
:1057C000F1001092F100D1C0282F2D7F09F0F4C014
:1057D000882319F0823061F0EFC080911B03813083
:1057E00009F0EAC0933009F080E0809316032EC0E0
:1057F00080911B0381112AC080911D038F702FEFB0
:10580000280F263008F0D8C08093E9002091EB00E3
:1058100020FF1CC0933021F48091EB00806214C003
:105820009091EB0090619093EB0021E030E0A901B2
:1058300002C0440F551F8A95E2F74093EA00109288
:10584000EA008091EB0088608093EB001092E90001
:105850008091E800877F8093E8000E94B129ACC066
:105860008111AAC010911B031F778091E3008078FB
:10587000812B8093E3008091E800877F8093E8008C
:105880000E94B1298091E80080FFFCCF8091E30065
:1058900080688093E300111102C082E001C083E0C0
:1058A0008093180389C08058823008F085C08091A9
:1058B0001B0390911C038C3D53E0950779F583E021
:1058C0008A838AE289834FB7F894DE01139620E039
:1058D0003EE051E2E32FF0E050935700E49120FFC7
:1058E00003C0E295EF703F5FEF708E2F90E0EA30DB
:1058F00010F0C79601C0C0968D939D932F5F243101
:1059000049F74FBF8091E800877F8093E8006AE203
:1059100070E0CE0101960E94BD2816C060911D0363
:1059200070911E03AE014F5F5F4F0E940428BC01BF
:10593000892B09F441C09091E800977F9093E8008B
:1059400089819A810E941B298091E8008B7780933E
:10595000E80032C0803881F58091E800877F80932D
:10596000E800809114038093F1008091E8008E7725
:1059700072CF811121C080911B0390911C03992744
:105980000297D4F48091E800877F8093E8008091AB
:105990001B03809314030E94B12980911403811189
:1059A00006C08091E30087FD02C081E001C084E071
:1059B000809318030E9482268091E80083FF0AC02A
:1059C0008091E800877F8093E8008091EB008062FF
:1059D0008093EB00AA960FB6F894DEBF0FBECDBF42
:1059E000DF91CF911F910895CF9380911803882361
:1059F000A1F0C091E900CF709091EC00892F8170E7
:105A000090FD80E8C82B1092E9008091E80083FDAA
:105A10000E94942BCF70C093E900CF910895991BF9
:105A200079E004C0991F961708F0961B881F7A9595
:105A3000C9F78095089597FB072E16F4009407D0B8
:105A400077FD09D00E94352D07FC05D03EF49095D6
:105A500081959F4F0895709561957F4F0895EE0F42
:105A6000FF1F0590F491E02D0994AA1BBB1B51E187
:105A700007C0AA1FBB1FA617B70710F0A61BB70BBE
:105A8000881F991F5A95A9F780959095BC01CD0163
:105A90000895FB01DC0104C08D910190801921F46F
:105AA00041505040C8F7881B990B0895F999FECFD3
:105AB00092BD81BDF89A992780B50895A8E1B0E01C
:105AC00042E050E00C948A2D262FF999FECF92BD2A
:105AD00081BDF89A019700B4021639F01FBA20BDB3
:105AE0000FB6F894FA9AF99A0FBE08950396272FE5
:105AF0000E94652D0E94642D252F0E94652D242F64
:105B00000C94652D0196272F0E94652D0C94642D11
:105B1000DC01CB01FC01F999FECF06C0F2BDE1BD6D
:105B2000F89A319600B40D9241505040B8F708955C
:045B3000F894FFCF17
:105B3400C8007A02280850011E0A14017125942510
:105B4400752504260026742501E200E900EA00B563
:105B540000B600B700CD008301CC008A0192019405
:105B6400012102230224022502260227022A02B36B
:105B740000B4006F007000818283E200E900EA0053
:105B8400B500B600B700CD008301CC008A019201B4
:105B940094012102230224022502260227022A025A
:105BA400B300B4006F00700081828397663534C6F9
:105BB4009436F6F79637909193923F3F3F006D6B82
:105BC4005F64656C6179006D6B5F696E7465727694
:105BD400616C006D6B5F6D61785F73706565640007
:105BE4006D6B5F74696D655F746F5F6D6178006D77
:105BF4006B5F776865656C5F6D61785F7370656511
:105C040064006D6B5F776865656C5F74696D655F73
:105C1400746F5F6D61780040B622A60CF00BCE0B5A
:065C2400730B8C0BA50BB5
:00000001FF
